:101A240033302E322020200008000803080608095D
:101A3400080C080F081208150819081C081F0822AA
:101A440008250828082B082F083208350838083BD1
:101A5400083E084108450848084B084E08510854F8
:101A64000857085B085E086108640867086A086D1F
:101A7400087108740877087A087D08800883088646
:101A8400088A088D0890089308960899089C08A06D
:101A940008A308A608A908AC08AF08B208B508B995
:101AA40008BC08BF08C208C508C808CB08CE08D2BD
:101AB40008D508D808DB08DE08E108E408E708EBE5
:101AC40008EE08F108F408F708FA08FD090009040B
:101AD4000907090A090D0910091309160919091C2E
:101AE4000920092309260929092C092F0932093556
:101AF4000938093C093F094209450948094B094E7F
:101B0400095109540957095B095E096109640967A8
:101B1400096A096D0970097309760979097D0980D3
:101B2400098309860989098C098F099209950998FD
:101B3400099B099E09A209A509A809AB09AE09B127
:101B440009B409B709BA09BD09C009C309C609C955
:101B540009CC09D009D309D609D909DC09DF09E27E
:101B640009E509E809EB09EE09F109F409F709FAAD
:101B740009FD0A000A030A060A090A0D0A100A13D3
:101B84000A160A190A1C0A1F0A220A250A280A2BFD
:101B94000A2E0A310A340A370A3A0A3D0A400A432D
:101BA4000A460A490A4C0A4F0A520A550A580A5B5D
:101BB4000A5E0A610A640A670A6A0A6D0A700A738D
:101BC4000A760A790A7C0A7F0A820A850A880A8BBD
:101BD4000A8E0A910A940A970A9A0A9D0AA00AA3ED
:101BE4000AA60AA90AAC0AAE0AB10AB40AB70ABA22
:101BF4000ABD0AC00AC30AC60AC90ACC0ACF0AD255
:101C04000AD50AD80ADB0ADE0AE10AE30AE60AE987
:101C14000AEC0AEF0AF20AF50AF80AFB0AFE0B01BB
:101C24000B040B070B090B0C0B0F0B120B150B18EA
:101C34000B1B0B1E0B210B240B260B290B2C0B2F20
:101C44000B320B350B380B3B0B3D0B400B430B4658
:101C54000B490B4C0B4F0B510B540B570B5A0B5D91
:101C64000B600B630B650B680B6B0B6E0B710B74CA
:101C74000B760B790B7C0B7F0B820B850B870B8A06
:101C84000B8D0B900B930B950B980B9B0B9E0BA141
:101C94000BA40BA60BA90BAC0BAF0BB10BB40BB77E
:101CA4000BBA0BBD0BBF0BC20BC50BC80BCA0BCDBC
:101CB4000BD00BD30BD60BD80BDB0BDE0BE10BE3FA
:101CC4000BE60BE90BEB0BEE0BF10BF40BF60BF93C
:101CD4000BFC0BFF0C010C040C070C090C0C0C0F77
:101CE4000C120C140C170C1A0C1C0C1F0C220C24B8
:101CF4000C270C2A0C2D0C2F0C320C350C370C3AFB
:101D04000C3D0C3F0C420C450C470C4A0C4C0C4F40
:101D14000C520C540C570C5A0C5C0C5F0C620C6487
:101D24000C670C690C6C0C6F0C710C740C770C79CF
:101D34000C7C0C7E0C810C840C860C890C8B0C8E18
:101D44000C900C930C960C980C9B0C9D0CA00CA264
:101D54000CA50CA80CAA0CAD0CAF0CB20CB40CB7AF
:101D64000CB90CBC0CBE0CC10CC30CC60CC90CCBFE
:101D74000CCE0CD00CD30CD50CD80CDA0CDD0CDF4B
:101D84000CE20CE40CE70CE90CEB0CEE0CF00CF39D
:101D94000CF50CF80CFA0CFD0CFF0D020D040D07EC
:101DA4000D090D0B0D0E0D100D130D150D180D1A3B
:101DB4000D1C0D1F0D210D240D260D280D2B0D2D91
:101DC4000D300D320D340D370D390D3C0D3E0D40E7
:101DD4000D430D450D470D4A0D4C0D4E0D510D5340
:101DE4000D560D580D5A0D5D0D5F0D610D640D6698
:101DF4000D680D6A0D6D0D6F0D710D740D760D78F6
:101E04000D7B0D7D0D7F0D810D840D860D880D8A52
:101E14000D8D0D8F0D910D940D960D980D9A0D9DB0
:101E24000D9F0DA10DA30DA50DA80DAA0DAC0DAE12
:101E34000DB10DB30DB50DB70DB90DBC0DBE0DC073
:101E44000DC20DC40DC60DC90DCB0DCD0DCF0DD1D9
:101E54000DD30DD60DD80DDA0DDC0DDE0DE00DE23F
:101E64000DE50DE70DE90DEB0DED0DEF0DF10DF3A6
:101E74000DF50DF70DFA0DFC0DFE0E000E020E040D
:101E84000E060E080E0A0E0C0E0E0E100E120E1476
:101E94000E160E180E1B0E1D0E1F0E210E230E25E0
:101EA4000E270E290E2B0E2D0E2F0E310E330E354E
:101EB4000E370E390E3B0E3C0E3E0E400E420E44C3
:101EC4000E460E480E4A0E4C0E4E0E500E520E5436
:101ED4000E560E580E5A0E5B0E5D0E5F0E610E63AB
:101EE4000E650E670E690E6B0E6C0E6E0E700E7222
:101EF4000E740E760E780E790E7B0E7D0E7F0E819B
:101F04000E830E840E860E880E8A0E8C0E8E0E8F15
:101F14000E910E930E950E960E980E9A0E9C0E9E92
:101F24000E9F0EA10EA30EA50EA60EA80EAA0EAC11
:101F34000EAD0EAF0EB10EB20EB40EB60EB80EB993
:101F44000EBB0EBD0EBE0EC00EC20EC30EC50EC716
:101F54000EC80ECA0ECC0ECD0ECF0ED10ED20ED49C
:101F64000ED60ED70ED90EDB0EDC0EDE0EDF0EE122
:101F74000EE30EE40EE60EE70EE90EEA0EEC0EEEAC
:101F84000EEF0EF10EF20EF40EF50EF70EF90EFA38
:101F94000EFC0EFD0EFF0F000F020F030F050F06C0
:101FA4000F080F090F0B0F0C0F0E0F0F0F110F124D
:101FB4000F140F150F160F180F190F1B0F1C0F1EE0
:101FC4000F1F0F210F220F230F250F260F280F2974
:101FD4000F2A0F2C0F2D0F2F0F300F310F330F340B
:101FE4000F350F370F380F3A0F3B0F3C0F3E0F3FA3
:101FF4000F400F420F430F440F450F470F480F493F
:102004000F4B0F4C0F4D0F4F0F500F510F520F54DA
:102014000F550F560F570F590F5A0F5B0F5C0F5E7A
:102024000F5F0F600F610F620F640F650F660F671C
:102034000F680F6A0F6B0F6C0F6D0F6E0F6F0F71C0
:102044000F720F730F740F750F760F770F790F7A66
:102054000F7B0F7C0F7D0F7E0F7F0F800F810F8210
:102064000F840F850F860F870F880F890F8A0F8BB8
:102074000F8C0F8D0F8E0F8F0F900F910F920F9368
:102084000F940F950F960F970F980F990F9A0F9B18
:102094000F9C0F9D0F9E0F9F0FA00FA10FA20FA3C8
:1020A4000FA40FA50FA50FA60FA70FA80FA90FAA7E
:1020B4000FAB0FAC0FAD0FAE0FAE0FAF0FB00FB134
:1020C4000FB20FB30FB40FB40FB50FB60FB70FB8ED
:1020D4000FB90FB90FBA0FBB0FBC0FBD0FBD0FBEA9
:1020E4000FBF0FC00FC10FC10FC20FC30FC40FC466
:1020F4000FC50FC60FC70FC70FC80FC90FCA0FCA26
:102104000FCB0FCC0FCC0FCD0FCE0FCE0FCF0FD0E8
:102114000FD00FD10FD20FD20FD30FD40FD40FD5AE
:102124000FD60FD60FD70FD80FD80FD90FD90FDA74
:102134000FDB0FDB0FDC0FDC0FDD0FDD0FDE0FDF3E
:102144000FDF0FE00FE00FE10FE10FE20FE20FE30B
:102154000FE30FE40FE40FE50FE50FE60FE60FE7DB
:102164000FE70FE80FE80FE90FE90FEA0FEA0FEBAB
:102174000FEB0FEC0FEC0FEC0FED0FED0FEE0FEE7E
:102184000FEF0FEF0FEF0FF00FF00FF00FF10FF154
:102194000FF20FF20FF20FF30FF30FF30FF40FF42C
:1021A4000FF40FF50FF50FF50FF60FF60FF60FF707
:1021B4000FF70FF70FF70FF80FF80FF80FF80FF9E5
:1021C4000FF90FF90FF90FFA0FFA0FFA0FFA0FFBC5
:1021D4000FFB0FFB0FFB0FFB0FFC0FFC0FFC0FFCA7
:1021E4000FFC0FFD0FFD0FFD0FFD0FFD0FFD0FFD8C
:1021F4000FFE0FFE0FFE0FFE0FFE0FFE0FFE0FFE73
:102204000FFF0FFF0FFF0FFF0FFF0FFF0FFF0FFF5A
:102214000FFF0FFF0FFF0FFF0FFF0FFF0FFF0FFF4A
:102224000FFF0FFF0FFF0FFF0FFF0FFF0FFF0FFF3A
:102234000FFF0FFF0FFF0FFF0FFF0FFF0FFF0FFF2A
:102244000FFF0FFF0FFF0FFF0FFF0FFF0FFF0FFF1A
:102254000FFF0FFE0FFE0FFE0FFE0FFE0FFE0FFE11
:102264000FFE0FFD0FFD0FFD0FFD0FFD0FFD0FFD09
:102274000FFC0FFC0FFC0FFC0FFC0FFB0FFB0FFB05
:102284000FFB0FFB0FFA0FFA0FFA0FFA0FF90FF902
:102294000FF90FF90FF80FF80FF80FF80FF70FF702
:1022A4000FF70FF70FF60FF60FF60FF50FF50FF503
:1022B4000FF40FF40FF40FF30FF30FF30FF20FF209
:1022C4000FF20FF10FF10FF00FF00FF00FEF0FEF10
:1022D4000FEF0FEE0FEE0FED0FED0FEC0FEC0FEC19
:1022E4000FEB0FEB0FEA0FEA0FE90FE90FE80FE826
:1022F4000FE70FE70FE60FE60FE50FE50FE40FE436
:102304000FE30FE30FE20FE20FE10FE10FE00FE045
:102314000FDF0FDF0FDE0FDD0FDD0FDC0FDC0FDB58
:102324000FDB0FDA0FD90FD90FD80FD80FD70FD66D
:102334000FD60FD50FD40FD40FD30FD20FD20FD186
:102344000FD00FD00FCF0FCE0FCE0FCD0FCC0FCCA1
:102354000FCB0FCA0FCA0FC90FC80FC70FC70FC6BD
:102364000FC50FC40FC40FC30FC20FC10FC10FC0DD
:102374000FBF0FBE0FBD0FBD0FBC0FBB0FBA0FB900
:102384000FB90FB80FB70FB60FB50FB40FB40FB323
:102394000FB20FB10FB00FAF0FAE0FAE0FAD0FAC4A
:1023A4000FAB0FAA0FA90FA80FA70FA60FA50FA574
:1023B4000FA40FA30FA20FA10FA00F9F0F9E0F9D9D
:1023C4000F9C0F9B0F9A0F990F980F970F960F95CD
:1023D4000F940F930F920F910F900F8F0F8E0F8DFD
:1023E4000F8C0F8B0F8A0F890F880F870F860F852D
:1023F4000F840F820F810F800F7F0F7E0F7D0F7C64
:102404000F7B0F7A0F790F770F760F750F740F7399
:102414000F720F710F6F0F6E0F6D0F6C0F6B0F6AD2
:102424000F680F670F660F650F640F620F610F600F
:102434000F5F0F5E0F5C0F5B0F5A0F590F570F564C
:102444000F550F540F520F510F500F4F0F4D0F4C8C
:102454000F4B0F490F480F470F450F440F430F42CF
:102464000F400F3F0F3E0F3C0F3B0F3A0F380F3713
:102474000F350F340F330F310F300F2F0F2D0F2C5B
:102484000F2A0F290F280F260F250F230F220F21A4
:102494000F1F0F1E0F1C0F1B0F190F180F160F15F0
:1024A4000F140F120F110F0F0F0E0F0C0F0B0F093C
:1024B4000F080F060F050F030F020F000EFF0EFD8E
:1024C4000EFC0EFA0EF90EF70EF50EF40EF20EF1E6
:1024D4000EEF0EEE0EEC0EEA0EE90EE70EE60EE43B
:1024E4000EE30EE10EDF0EDE0EDC0EDB0ED90ED790
:1024F4000ED60ED40ED20ED10ECF0ECD0ECC0ECAE9
:102504000EC80EC70EC50EC30EC20EC00EBE0EBD43
:102514000EBB0EB90EB80EB60EB40EB20EB10EAF9F
:102524000EAD0EAC0EAA0EA80EA60EA50EA30EA1FD
:102534000E9F0E9E0E9C0E9A0E980E960E950E935E
:102544000E910E8F0E8E0E8C0E8A0E880E860E84C1
:102554000E830E810E7F0E7D0E7B0E790E780E7625
:102564000E740E720E700E6E0E6C0E6B0E690E678C
:102574000E650E630E610E5F0E5D0E5B0E5A0E58F5
:102584000E560E540E520E500E4E0E4C0E4A0E485F
:102594000E460E440E420E400E3E0E3C0E3B0E39CD
:1025A4000E370E350E330E310E2F0E2D0E2B0E2937
:1025B4000E270E250E230E210E1F0E1D0E1B0E18A8
:1025C4000E160E140E120E100E0E0E0C0E0A0E081F
:1025D4000E060E040E020E000DFE0DFC0DFA0DF794
:1025E4000DF50DF30DF10DEF0DED0DEB0DE90DE70F
:1025F4000DE50DE20DE00DDE0DDC0DDA0DD80DD686
:102604000DD30DD10DCF0DCD0DCB0DC90DC60DC400
:102614000DC20DC00DBE0DBC0DB90DB70DB50DB37A
:102624000DB10DAE0DAC0DAA0DA80DA50DA30DA1F8
:102634000D9F0D9D0D9A0D980D960D940D910D8F76
:102644000D8D0D8A0D880D860D840D810D7F0D7DF8
:102654000D7B0D780D760D740D710D6F0D6D0D6A7A
:102664000D680D660D640D610D5F0D5D0D5A0D58FD
:102674000D560D530D510D4E0D4C0D4A0D470D4584
:102684000D430D400D3E0D3C0D390D370D340D320B
:102694000D300D2D0D2B0D280D260D240D210D1F94
:1026A4000D1C0D1A0D180D150D130D100D0E0D0B1F
:1026B4000D090D070D040D020CFF0CFD0CFA0CF8AE
:1026C4000CF50CF30CF00CEE0CEB0CE90CE70CE441
:1026D4000CE20CDF0CDD0CDA0CD80CD50CD30CD0CE
:1026E4000CCE0CCB0CC90CC60CC30CC10CBE0CBC60
:1026F4000CB90CB70CB40CB20CAF0CAD0CAA0CA8F2
:102704000CA50CA20CA00C9D0C9B0C980C960C9385
:102714000C900C8E0C8B0C890C860C840C810C7E1A
:102724000C7C0C790C770C740C710C6F0C6C0C69B0
:102734000C670C640C620C5F0C5C0C5A0C570C5448
:102744000C520C4F0C4C0C4A0C470C450C420C3FE1
:102754000C3D0C3A0C370C350C320C2F0C2D0C2A7A
:102764000C270C240C220C1F0C1C0C1A0C170C1418
:102774000C120C0F0C0C0C090C070C040C010BFFB5
:102784000BFC0BF90BF60BF40BF10BEE0BEB0BE95B
:102794000BE60BE30BE10BDE0BDB0BD80BD60BD3F9
:1027A4000BD00BCD0BCA0BC80BC50BC20BBF0BBD9B
:1027B4000BBA0BB70BB40BB10BAF0BAC0BA90BA63D
:1027C4000BA40BA10B9E0B9B0B980B950B930B90DF
:1027D4000B8D0B8A0B870B850B820B7F0B7C0B7984
:1027E4000B760B740B710B6E0B6B0B680B650B6329
:1027F4000B600B5D0B5A0B570B540B510B4F0B4CCF
:102804000B490B460B430B400B3D0B3B0B380B3575
:102814000B320B2F0B2C0B290B260B240B210B1E1D
:102824000B1B0B180B150B120B0F0B0C0B090B07C7
:102834000B040B010AFE0AFB0AF80AF50AF20AEF76
:102844000AEC0AE90AE60AE30AE10ADE0ADB0AD824
:102854000AD50AD20ACF0ACC0AC90AC60AC30AC0D0
:102864000ABD0ABA0AB70AB40AB10AAE0AAC0AA97E
:102874000AA60AA30AA00A9D0A9A0A970A940A9128
:102884000A8E0A8B0A880A850A820A7F0A7C0A79D8
:102894000A760A730A700A6D0A6A0A670A640A6188
:1028A4000A5E0A5B0A580A550A520A4F0A4C0A4938
:1028B4000A460A430A400A3D0A3A0A370A340A31E8
:1028C4000A2E0A2B0A280A250A220A1F0A1C0A1998
:1028D4000A160A130A100A0D0A090A060A030A004C
:1028E40009FD09FA09F709F409F109EE09EB09E808
:1028F40009E509E209DF09DC09D909D609D309D0B8
:1029040009CC09C909C609C309C009BD09BA09B76F
:1029140009B409B109AE09AB09A809A509A2099E20
:10292400099B099809950992098F098C09890986D7
:1029340009830980097D0979097609730970096D8C
:10294400096A096709640961095E095B0957095441
:102954000951094E094B094809450942093F093CF7
:10296400093809350932092F092C092909260923AF
:102974000920091C0919091609130910090D090A66
:1029840009070904090008FD08FA08F708F408F122
:1029940008EE08EB08E708E408E108DE08DB08D8DD
:1029A40008D508D208CE08CB08C808C508C208BF95
:1029B40008BC08B908B508B208AF08AC08A908A64D
:1029C40008A308A0089C0899089608930890088D05
:1029D400088A088608830880087D087A08770874BE
:1029E4000871086D086A086708640861085E085B76
:1029F400085708540851084E084B08480845084130
:102A0400083E083B083808350832082F082B0828E8
:102A140008250822081F081C081908150812080FA1
:102A2400080C0809080608031000100B10161021E2
:102A3400102C10371043104E105910651070107B75
:102A440010871092109E10A910B510C010CC10D889
:102A540010E310EF10FB11071113111E112A113688
:102A64001142114E115A11661172117E118A119779
:102A740011A311AF11BB11C811D411E011ED11F95B
:102A840012061212121F122B123812451251125E24
:102A9400126B127812841291129E12AB12B812C5E4
:102AA40012D212DF12EC12F9130613141321132E8F
:102AB400133C1349135613641371137F138C139A25
:102AC40013A713B513C313D013DE13EC13FA1408AE
:102AD400141614231431143F144E145C146A14781D
:102AE4001486149414A314B114BF14CE14DC14EB80
:102AF40014F91508151615251534154215511560C8
:102B0400156F157E158D159C15AB15BA15C915D8FD
:102B140015E715F616051615162416331643165220
:102B2400166216711681169016A016B016C016CF2E
:102B340016DF16EF16FF170F171F172F173F174F24
:102B4400175F17701780179017A117B117C117D205
:102B540017E217F3180418141825183618471857CD
:102B640018681879188A189B18AC18BE18CF18E082
:102B740018F119021914192519371948195A196B1A
:102B8400197D198F19A019B219C419D619E819FA9F
:102B94001A0C1A1E1A301A421A551A671A791A8B05
:102BA4001A9E1AB01AC31AD51AE81AFB1B0E1B2058
:102BB4001B331B461B591B6C1B7F1B921BA51BB88D
:102BC4001BCC1BDF1BF21C061C191C2D1C401C54A7
:102BD4001C671C7B1C8F1CA31CB71CCB1CDF1CF3A9
:102BE4001D071D1B1D2F1D431D581D6C1D801D958C
:102BF4001DA91DBE1DD31DE71DFC1E111E261E3B57
:102C04001E501E651E7A1E8F1EA41EB91ECF1EE402
:102C14001EFA1F0F1F251F3A1F501F661F7B1F918F
:102C24001FA71FBD1FD31FE90C000B000A000900DA
:102C3400080007000600050004000300020001006C
:042C4400010000008B
:10341E004102A74CC100C1024102A6004102A80010
:10342E00C1014102B50041029F014202A30001C148
:10343E0003C1044102A50642026400004102660077
:10344E004202B100014202B300004202A900004252
:0D345E0002A0000142026700004102A2012D
:1037D10053E3DF75B61043E32075AB80E4FF0FEFD1
:1037E100B414FB43ABC0E5AB30E5FB75A90275B280
:0137F1008750
:0137F20022B4
:1038F600758850758922758E04758C5C758D567524
:0E390600C804E4F5CA75CBFEF5CC75CDFE22E3
:1039EA0075BC909002A5E0F5BB75E88075BAF72220
:073A550075B9F675B5F62204
:043A7D00E4F5D12279
:10393100E4F5F275A48075A63875D40375D5FF75C5
:0B394100F3FFF5D675E10475E24022AB
:083A3D0043E608D2ADD2AB2232
:10391400E4F5881237D11239311238F61239EA1225
:0D3924003A55123A7D123A3DC2A5C2022268
:10128E00C20A53D9BF123914A2A2920A9002A730F1
:10129E000A05744CF08003744DF09002A7E0FF1223
:1012AE003A0743F601123998123738E580544090C8
:1012BE0002B5F0D2AF300308123095C2031238D700
:1012CE00300405120FBFC2047B017A0279B61219DF
:1012DE00E0EF60E19002B8E0120B4C135404139B44
:1012EE0005131614130816130F17131B1A133D1B91
:1012FE0013481D134E1E000013EBD201D20202132F
:10130E00EBC202C2010213EBD2000213EB7B017A95
:10131E000279B69002C6EBF0A3EAF0A3E9F0120947
:10132E009DFE9002A7E0FF6E60030213EB80059016
:10133E0002A7E0FF1238570213EB123A6A0213EBC0
:10134E00123A770213EB7B017A0279B69002C9EB5F
:10135E00F0A3EAF0A3E9F09000031209B6FF9002A1
:10136E00A7E06F707830016D9002C904F0A3EAF027
:10137E00A3E9F09000051209B6FF9000061209B617
:10138E00FD9000041209B6FB1231FB80487B017AF6
:10139E000279B69002C9EBF0A3EAF0A3E9F090004F
:1013AE00031209B6FF9002A7E06F7031300126904C
:1013BE0002C904F0A3EAF0A3E9F09000051209B601
:1013CE00FF9000061209B6FD9000041209B6FB123A
:1013DE00192A1237389002A7E0FF1238B8200103FD
:1013EE000212D69002B8E014603424FA60531470DE
:1013FE000302149D240660030212D61239D97B0112
:10140E007A0279B69002C6EBF0A3EAF0A3E9F09067
:10141E0000031209B6900333F0123A4D806B123965
:10142E00D97B017A0279B69002C6EBF0A3EAF0A35B
:10143E00E9F09000031209B6900333F012373880AA
:10144E00481239D97B017A0279B69002CCEBF0A31F
:10145E00EAF0A3E9F09000031209B6FF900004121F
:10146E0009B6FD9000051209B6FBC0039002CCE050
:10147E00FBA3E0FAA3E0F99000061209B69002E68B
:10148E00F0D003123149123738123A290212D6120D
:10149E0039D97B017A0279B69002CCEBF0A3EAF04F
:1014AE00A3E9F09000031209B6FF9000041209B6EA
:1014BE00FD9000051209B6FB12166D123738123A5E
:0414CE00290212D607
:1039C700A20292A5E50824FFB392A4E50824FF927A
:0239D700A32229
:103095009002B5E090029FF0E58054409002B5F0B3
:1030A500E07042C3900264E09408500EA3E004F07F
:1030B5007059900264E004F08051A200E433FF905F
:1030C5000266E070047E0180027E00EE5F600E9075
:1030D50002A7E0FF7BFF7A1A7924123492900266E8
:1030E5007401F08026E4900264F0A3F090029FE062
:1030F5007014900266E0700EE50870047F0180028E
:103105007F008F08D209E4900266F09002A6E09055
:1031150002A8F0E5A054029002A6F09002A8E06093
:10312500229002A6E0701C9002A8F020000C9003EB
:1031350033F0123A4DC209C20222A201B39201A292
:03314500019202F2
:013148002264
:031A0C000236950A
:10369500C0E0C0F0C083C082C0D075D000C000C0FB
:1036A50001C002C003C004C005C006C007122FA593
:1036B500D007D006D005D004D003D002D001D00069
:0B36C500D0D0D082D083D0F0D0E03213
:102FA5009002A9E0FEA3E0F5969002B3E0FCA3E051
:102FB500F5F4EEF597ECF5F59002A0E0FEA3E0FF41
:102FC500900268E02FF0900267E03EF0E0C4F8540C
:102FD500F0C868FEA3E0C4540F48FFEE540FFEE4AA
:102FE5002FFDEE3404540FFCC3EE64809488502109
:102FF500EF25E0FFEE33FE742C2FF582741A3EF5B3
:1030050083E493FF7401939002A9CFF0A3EFF080BE
:103015002BEE5407FEEF25E0FFEE33FE742C2FF563
:1030250082741A3EF583E493FE740193FFC374FF23
:103035009F9002AAF0740F9E9002A9F0C3EC6480E1
:1030450094885020ED25E0FFEC33FE742C2FF5829B
:10305500741A3EF583E493FF7401939002B3CFF0A5
:10306500A3EFF022EC5407FEED25E0FFEE33FE74EE
:103075002C2FF582741A3EF583E493FE740193FFB9
:0F308500C374FF9F9002B4F0740F9E9002B3F0DB
:013094002219
:031A120002365742
:10365700C0E0C0F0C083C082C0D075D000C000C039
:1036670001C002C003C004C005C006C00753C87F1D
:10367700123878D007D006D005D004D003D002D0B6
:0E36870001D000D0D0D082D083D0F0D0E0327D
:103878009002A5E0F5BBE004F0E0D36480948F40AB
:103888000B7406F01239C7123A5CD20443E81022CE
:073A5C00E50824FF92872218
:031A210002353E4D
:10353E00C0E0C083C082C0D075D000C004C005C03A
:03354E0006C007AD
:1035510053E8DFADBDAFBEEFFE7C00E42DFFEC3ED6
:10356100FEADBBED25E02469F582E43402F583EE7E
:06357100F0A3EFF0D2030D
:10357700D007D006D005D004D0D0D082D083D0E0F9
:013587003211
:100FBF00900283E0FFA3E09002ABCFF0A3EFF0909D
:100FCF000281E0FFA3E09002ADCFF0A3EFF090021B
:100FDF007FE0FFA3E09002AFCFF0A3EFF09002A26B
:100FEF00E060329002ABE0FFA3E0900366CFF0A386
:100FFF00EFF09002ADE0FFA3E0900368CFF0A3EF16
:10100F00F09002AFE0FFA3E090036ACFF0A3EFF000
:10101F00E49002A2F07F00120C9D7F01120C9D7FC5
:10102F0002120C9DAF0CAE0BD374649F74089E50CC
:10103F0009EF249CFFEE34F78022C3749C9F740742
:10104F009E5012C3EF9464EE94085009E49002D5B9
:10105F00F0A3F0800EEF2464FFEE34F89002D5F089
:10106F00A3EFF090027BE0FFA3E09002D9CFF0A3B3
:10107F00EFF0900279E0FEA3E0FFEE3395E0FDFC88
:10108F00E47B08FAF9F8123613E42FFFEE34FF90E1
:10109F0002DBF0A3EFF09002D5E0FEA3E0FBAA067F
:1010AF00EA3395E0F9F89002D9E0FEA3E0FFEE33C2
:1010BF0095E0FDFC120AAA9002CF120B0FE4FB7A07
:1010CF0008F9F89002CFE0FCA3E0FDA3E0FEA3E057
:1010DF00FF1236139002D3EEF0A3EFF0AE0DAF0E6A
:1010EF00E4FCFD9002DF120B0F9002DBE0FEA3E0A9
:1010FF00FFEE3395E0FDFC9002DFE0F8A3E0F9A3EB
:10110F00E0FAA3E0FB120AAA9002CF120B0FE4FB46
:10111F007A04F9F89002CFE0FCA3E0FDA3E0FEA370
:10112F00E0FF1236139002D7EEF0A3EFF0AE09AF47
:10113F000A7C007D09120A177D0C120A29EF24ABD5
:10114F00FFEE3402FE9002D4E02FFF9002D3E03E78
:10115F00FE9002A3F0A3EFF0D394FFEE6480948F80
:10116F00400A9002A3740FF0A374FFF0C39002A380
:10117F00E0648094805004E4F0A3F09002A3E0FEBA
:10118F00A3E0FFEE3395E0FDFCE4FB7A0DF9F812D6
:10119F000AAA9002CF120B0F9002CFE0FCA3E0FD42
:1011AF00A3E0FEA3E0FFE4FB7A10F9F812361390E8
:1011BF0002CF120B0FE49002D3F0A3F09002D4E011
:1011CF0025E0FF9002D3E033FE742C2FF582742CB0
:1011DF003EF583E493FE740193FF9002D5EEF0A3E6
:1011EF00EFF0EE3395E0FDFC9002CFE0F8A3E0F9CD
:1011FF00A3E0FAA3E0FBC3120AF940209002CFA3A9
:10120F00A3A3E0FF9002D5A3E0FEEF9E9002DDF0D6
:10121F009002D3A3E0049002DEF0801A9002D4E093
:10122F0004F070069002D3E004F09002D3E0700453
:10123F00A3E0640D70869002DDE075F002A4242C0B
:10124F00F582E5F0342AF583E493FE740193FF9061
:10125F0002DEE0FDEFA805088005CEC313CE13D83C
:10126F00F9FF9002A0EEF0A3EFF09002D7E0FEA3FB
:0E127F00E0FF9002A1E02FF09002A0E03EF010
:01128D00223E
:10381500A2AFE433FCC2AF758F0175B7A575B7F1DB
:103825008F828E83EDF0E4F58FAF04EF24FF92AF26
:013835002270
:10389800A2AFE433FDC2AF758F0375B7A575B7F155
:0F38A8008F828E83E4F0F58FAF05EF24FF92AF90
:0138B70022EE
:1034F20090036CEEF0A3EFF0A3ECF0A3EDF0EB4A37
:10350200603990036CE0FEA3E0FFA3E0FCA3E0F5CA
:10351200828C83E0FD123815EB1B70011A90036F49
:10352200E004F0700690036EE004F090036DE00496
:0C353200F070CB90036CE004F080C3222A
:083A4500E4900000F0A3F02260
:10376300900000E0FEA3E0FF123898900000E0FE16
:10377300A3E0FF7C007D027B007A021234F2E49026
:063783000000F0A3F0229B
:0A329000A90590035AEEF0A3EFF039
:10329A00EE54FEFE900000E0FCA3E0FD7002EE6C2E
:1032AA006057ED4C600312376390035AE0FEEE5408
:1032BA00FEFE7F00900000F0A3EFF090035CEEF0BA
:1032CA00A3EFF0A37400F0A37402F07E0290035CF3
:1032DA00E475F001120A9485F082F583E493FD9077
:1032EA00035EE475F001120A9485F082F583EDF02D
:1032FA00EF1F70011EEF4E70D490035AE0FCA3E05A
:10330A00FDEC5401FC74022DF58274003CF583E94E
:01331A00F0C2
:01331B00228F
:1035880090034CEEF0A3EFF0A3EBF0A3EAF0A3E96D
:10359800F090035174FFF5F0120A9445F0602690FC
:1035A800034CE475F001120A94AFF0FE90034EE06C
:1035B800FBA3E475F001120A94A9F0FA12099DFD23
:0635C80012329080CC22BB
:073A630043C14053E6FE22BF
:1017DB00900318E0FFA3E0FCA3E0FDA3E0FBA3E074
:1017EB00FAA3E0F99002F5E50FF0E510A3F09003F2
:0617FB0020E09002F7F06F
:101801009002EFEFF0A3ECF0A3EDF0A3EBF0A3EA6D
:04181100F0A3E9F067
:101815009002F87403F0A374E8F0E5C120E5FBD26B
:10182500C1C2C4D2C5E4FF90038AF030C0FDE5C053
:1018350054FE244070030218D824FE602424E2607C
:101845000924FE600524E20218E0C2C5EF60030228
:1018550018E69002EFE025E044A0F5C27F030218E8
:10186500E6EFB4030A9002F0E0F5C27F058072EF5F
:10187500B4050B9002F0A3E0F5C27F068063EF6428
:1018850006703E9002F7E09002F2700FE0FBA3E4D1
:1018950075F001120A94A9F0FA8008E0FBA3E0FABA
:1018A500A3E0F912099DF5C29002F6E024FFF0903D
:1018B50002F5E034FFF0E07002A3E070247F0780BA
:1018C50020EFB40706D2C47F09801690038A7405F9
:1018D500F0800E90038A7402F0800690038A7401EA
:1018E500F0EFB40904C2C0803690038AE0FE6406B6
:1018F5006012EEB402169002F874FFF5F0120A7E3B
:1019050045F06008D2C5E490038AF0FF90038AE0B1
:101915006008C2C5D2C4C2C08005C2C0021830E585
:04192500C120E5FBFD
:01192900229B
:102C48009002FAEFF0A3ECF0A3EDF0A3EBF0A3EA07
:042C5800F0A3E9F00C
:102C5C009003027403F0A374E8F0E5C120E5FBD205
:102C6C00C1C2C4D2C5E4FF90038AF030C0FDE5C0F8
:102C7C0054FE24C87003022D3924AE607A24CA7025
:102C8C0003022D4124FE603824E2600924FE600515
:102C9C0024E2022D49C2C5EF700F9002FAE025E044
:102CAC0044A0F5C27F03022D4FEF64016003022D97
:102CBC004F9002FAE025E044A1F5C27F04022D4FAB
:102CCC00EFB4030A9002FBE0F5C27F058075EFB408
:102CDC00050B9002FBA3E0F5C27F068066EFB406FD
:102CEC0006D2C57F01805CEFB404047F028054904F
:102CFC00038A7405F0804C9002FDE0FBA3E475F0B0
:102D0C0001120A94A9F0FAE5C21209E3900301E05A
:102D1C0024FFF0900300E034FFF0E07002A3E070B9
:102D2C00087F09C2C1D2C4801A7F02801690038A20
:102D3C007406F0800E90038A7402F0800690038A69
:102D4C007401F0EFB40904C2C0803690038AE0FE2F
:102D5C0064066012EEB4021690030274FFF5F012D2
:102D6C000A7E45F06008D2C5E490038AF0FF900318
:102D7C008AE06008C2C5D2C4C2C08005C2C0022CA1
:062D8C0077E5C120E5FB24
:012D9200221E
:102E9E00900318EFF090031BEBF0A3EAF0A3E9F018
:082EAE00900319ECF0A3EDF014
:102EB600751100543FF512543F605CC3744095127F
:102EC600FFE49511FE90031EE0FCA3E0FDC39FEC1A
:102ED6009E50068C0F8D1080048E0F8F101217DBFC
:102EE60090038AE060037F022290031AE02510F027
:102EF600900319E0350FF0900320E0700B90031C4F
:102F0600E50F8510F0120A7EC390031FE09510F0BE
:102F160090031EE0950FF090031EE0F50FA3E0F579
:102F260010D3E5109400E50F94004070E51094402E
:102F3600E50F940050131217DB90038AE060037FBD
:102F46000222E4F50FF51080D8900318E0FFA3E005
:102F5600FCA3E0FDA3E0FBA3E0FAA3E0F99002F5F1
:102F6600E4F074401217F790038AE060037F0222B0
:102F760074C02510F51074FF350FF50F90031AE095
:102F86002440F0900319E03400F0900320E07091A3
:0E2F960090031C75F040120A7E022F277F0068
:012FA400220A
:1039B000900300E4F0A304F0122C4890038AE06026
:0739C000037F01227F0022BA
:10394C00900389EBF07B017A03798990031EE4F0F4
:0A395C00A304F0E4A3F0122E9E2253
:1037F300C007900342E0FFA3E0900300CFF0A3EFE4
:10380300F0D007122C4890038AE060037F01227FE7
:02381300002291
:10396600C00790034AE0FFA3E090031ECFF0A3EF49
:0A397600F0E4A3F0D007122E9E2209
:10346B00420262000042020D00004202080000C14D
:05347B0007C106C105B8
:0A3A1F00C206C207E490020CF02278
:1037AE00E4900262F0A3F090020DF0A3F0A3F0906B
:1037BE000208F0A3F0900203F0A37440F0E490022C
:0337CE000BF022DB
:061A1B00123A1F0237AE73
:0D39FA0075C19043E60190020A7401F022AD
:1039D90043C140E5C120E5FB121A1BE490020AF03D
:0139E90022BB
:0A3A290053C1BF90020A7401F0229D
:0D3A0700AE071239FA900207EEF0021A1B0A
:10378900E4900387F0A3F0300602FF222007FDD260
:1037990006900205E4F0A37410F0900250EFF0E4F3
:0437A900A3F07F0109
:0137AD0022F9
:1036D00030060A900205E07002A3E070037F00222A
:1036E000900206E024FFF0900205E034FFF0900223
:1036F00051E0FE04F074522EF582E43402F583EFBB
:04370000F07F012233
:0B3A1400300607C206D207123A332228
:0A3A3300E5C120E5FBC2C4D2C522A4
:1033A500900354EBF0A3EAF0A3E9F090020AE07071
:1033B50002FF22900357E0FE6005D3941040037F7F
:0833C5000022123789EF604E6F
:1033CD00E4900359F0900357E0FF900359E0FEC3DA
:1033DD009F5024900354E0FBA3E0FAA3E0F98E8202
:1033ED007583001209B6FF1236D0EF7002FF2290DE
:1033FD000359E004F080CEE490020CF0123A1490E0
:0E340D000358E070032007FD90020CE0FF2240
:03341B007FFF220E
:0E2D9300900370EBF0A3EAF0A3E9F0A3EDF0DB
:102DA100E4FFD3900263E09400900262E0648094B7
:102DB1008050012253E6FE900208E0FEA3E0240FBA
:102DC100F58274023EF583E0FF900208E475F0019C
:102DD100120A7EFCE5F064404C7006900208F0A3F4
:102DE100F0900204E004F07006900203E004F0E4C5
:102DF100FE900373E0FDEEC39D5054EEC39F504F10
:102E0100900208E0FCA3E0240FF58274023CF583F4
:102E1100E0FD900370E0FBA3E0FAA3E0F98E827578
:102E21008300ED1209F5900208E475F001120A7EA3
:102E3100FCE5F064404C7006900208F0A3F09002AB
:102E410004E004F07006900203E004F00E80A2EEAC
:102E5100C39F5029900208E475F001120A7EFCE537
:102E6100F064404C7006900208F0A3F0900204E078
:102E710004F07006900203E004F00E80D290026329
:102E8100E024FFF0900262E034FFF043E60190039A
:0C2E910073E0FEEFC39E50028002AF060B
:012E9D002212
:10398000D3900263E09400900262E06480948040EF
:08399000047F0180027F002288
:031A18000214D2E3
:1014D200C0E0C0F0C083C082C0D075D000C000C0E0
:0314E20006C0073A
:1014E500C20BE5C054FE120B4C15C10815C10A15F7
:1014F500880C15880E163A10163A12158E22159973
:101505002815992A158E2C158E2E157BC01534C2DB
:10151500151FE0151FE200001645C205900250E0B8
:10152500F5C2C2C5C2C490024F74FFF002164790BF
:10153500024FE0FFB4FF12900251E0F5C2C2C5C2EE
:10154500C490024FE4F0021647900251E0FEEFC34B
:101555009E501790024FE0FF04F074522FF582E47D
:101565003402F583E0F5C2021647D2C490020CE4BA
:10157500F0C20702164790020C74FDF0D2C5C2C432
:1015850002164790024F74FFF0D205C2C4C2C1D201
:10159500C5021647E5C26007900207E0B5C20E9086
:1015A5000202E4F0C2C5C2C4D2C1021647C2C4C217
:1015B500C130050302163FC2C5021647900202E07C
:1015C5007020E5C2F0E0FFC3900204E09F7480F84C
:1015D500900203E064809850031237AE900202E057
:1015E50004F0900204E024FFF0900203E034FFF0E1
:1015F50090020DE0FEA3E0240FF58274023EF58310
:10160500E5C2F090020DE475F001120A7EFEE5F0E8
:1016150064404E700690020DF0A3F0900202E014B3
:10162500F0700E900263E004F07006900262E00430
:10163500F0D2C1800DC2C4300508C205D2C58002F2
:10164500D20B300B1053C17F43C180C2C5C2C4C287
:07165500C1C20BC207C2C0B5
:10165C00D007D006D000D0D0D082D083D0F0D0E04C
:01166C00324B
:053A7100E5C15420FF37
:013A7600222D
:0E35CE00900360EBF0A3EAF0A3E9F0A3EDF0A8
:1035DC00E4900365F0900360E0FBA3E0FAA3E0F94C
:1035EC00A3E0900357F0900364E0900358F0E4FFDD
:1035FC001233A5EFB4FF0D900365E0FE04F0EEC3AB
:06360C00940340D17E0092
:013612002295
:0B19E000900384EBF0A3EAF0A3E9F011
:1019EB007E007F007D10120BA3900384E0FBA3E02D
:1019FB00FAA3E0F97D10122D93EF7002FF227F0105
:011A0B0022B8
:103492009003047422F0A3EFF0A37413F012099DB9
:1034A200900307F09000011209B6900308F0900013
:1034B200021209B6900309F09000031209B69003B4
:1034C2000AF09000041209B690030BF09000051266
:1034D20009B690030CF09000061209B690030DF0A5
:1034E2007B017A037904E4900364F07D0A0235CE0D
:103836009003747422F0A3EFF0A37403F0A374FF53
:10384600F07B017A037974E4900364F07D04023519
:01385600CEA3
:103857009003787422F0A3EFF0A3741CF0A374FF15
:10386700F07B017A037978E4900364F07D040235F4
:01387700CE82
:1038B800E490037CF0A3EFF0A3740AF0A3EFF07B8D
:0F38C800017A03797CE4900364F07D040235CE2D
:08348000C108C10941033B0032
:063A7700E490033BF02285
:073A6A0090033B7401F02200
:10331C00E4900381F0A37403F0E4A3F0FE7F07FDB7
:10332C00FB7A007908120BA3750B08750C00123A86
:10333C00457E7A7F017B017A037982900351E4F018
:10334C00A304F0123588E4900380F0900380E0FF32
:10335C00C3941E5029EF75F007A42402F582E434BF
:10336C007AAF82FE7B007A007908900351E4F0A3D7
:10337C007407F0123588900380E004F080CD12378A
:10338C00637E7A7F007B017A037983900351E4F0AA
:09339C00A304F012358802376326
:1038D70030091B200002D202300113200810900388
:0F38E7003BE070089002A7E0FF123836D20822AB
:10399800907A00E493F46007A3E49364036003124D
:0839A800331CE4900333F0220C
:10373800900333E0FFC3941E5020EF75F007A424D4
:1037480002F9747A35F0FA7BFF78087C007D007EF8
:0B375800007F07120977C209C2082297
:10370400900333E0C3941E502A123A45900333E0E9
:1037140075F007A42402F582E4347AAF82FE7B00BC
:103724007A007908900351E4F0A37407F012358805
:0437340012376322C3
:083A4D00123704C209C208226D
:053149009002E4EDF02E
:10314E009002E6E004F09002E9EFF0A3EBF09002BB
:10315E00E4E0FF9002E9E0FED39F40030231FAEE75
:10316E0075F007A42402F582E4347AAF829002EB64
:10317E00F0A3EFF09002EAE075F007A42402F582C6
:10318E00E4347AAF829002EDF0A3EFF0E49002E720
:10319E00F0A3F09002EDE475F001120A94AFF0FE88
:1031AE009002EBE0FCA3E0F5828C83E493FD1232F7
:1031BE00909002ECE004F070069002EBE004F090C8
:1031CE0002E8E004F070069002E7E004F0C390021B
:1031DE00E8E094079002E7E0940040B7123763905E
:0C31EE0002E9E004F0A3E004F002315C10
:0131FA0022B2
:05166D00900321EDF0E7
:10167200900326EFF0A3EBF0900321E0FF90032606
:10168200E0D39F40030217DAA3E075F007A4240217
:10169200F582E4347AAF82900322F0A3EFF0E49073
:1016A2000328F0A3F0900328E0FEA3E0FFC3940711
:1016B200EE94005038900322E0FCA3E0F5828C8384
:1016C200E493FD74342FF582E43403F583EDF09056
:1016D2000323E004F07006900322E004F090032953
:1016E200E004F070C0900328E004F080B890032674
:1016F200E075F007A42402F582E4347AAF82900305
:1017020024F0A3EFF0900327E075F007A42402F57C
:1017120082E4347AAF82900322F0A3EFF0E49003E4
:1017220028F0A3F0900322E475F001120A94AFF0BE
:10173200FE900324E0FCA3E0F5828C83E493FD1287
:101742003290900325E004F07006900324E004F048
:10175200900329E004F07006900328E004F0C3909F
:101762000329E09407900328E0940040B7900326F1
:10177200E075F007A42402F582E4347AAF82900384
:1017820024F0A3EFF0E4900328F0A3F0900328E004
:10179200FCA3E0FDC39407EC9400502C900324E4D6
:1017A20075F001120A94AFF0FE74342DF582E43420
:1017B20003F583E0FD123290900329E004F070CC2F
:1017C200900328E004F080C4123763900326E004FB
:0817D200F0A3E004F002167A16
:0117DA0022EC
:0B192A0090030EEFF0A3EDF0A3EBF034
:10193500A2AFE433A3F0C2AF123A6390030FE0FE07
:1019450090030EE0FDEDFF900316EEF0A3EFF0E43B
:10195500900312F0900310E0FF900316E0FCA3E063
:10196500FD7B017A037934900342E4F0A37407F018
:101975001237F3900317E02407F0900316E03400C4
:10198500F0900312E075F007A42402F9747A35F09B
:10199500FAA374FFF0A3EAF0A3E9F0123A45900325
:1019A50013A3E0FAA3E0AE02FF7B017A037934903A
:1019B5000351E4F0A37407F01235881237639003DE
:1019C50012E004F0E0C3941E408A9002A7E0FF12E3
:0A19D5003A07900311E024FF92AFDF
:0119DF0022E5
:0B31FB0090032AEFF0A3EDF0A3EBF02F
:10320600A2AFE433A3F0C2AF123A6390032BE0FE01
:1032160090032AE0FDEDFF90032FEEF0A3EFF0E41C
:1032260090032EF090032EE0FFC3941E504BEF75D3
:10323600F007A42402F582E4347AAF82FE900331CB
:10324600F0FAA3EFF0FB90032CE0FF90032FE0FCD5
:10325600A3E0FDA9037BFF90034AE4F0A37407F003
:10326600123966900330E02407F090032FE0340013
:10327600F090032EE004F080AB9002A7E0FF123A34
:093286000790032DE024FF92AF34
:01328F00221C
:093488004603660000000000008C
:0E0C9D0090FFFF120B72EFF090FFEE120B7241
:100CAB00851383851482E4F0A3F0900012120B9647
:100CBB00E025E02466F582E43403F583E0FEA3E04F
:100CCB00FFFBAA06E4F9F8900012120B96E075F000
:100CDB0002A424ABF582E5F03402F583E0FEA3E039
:100CEB00FFC3EF9BFFEE9AFEE499FDE498FC85139E
:100CFB0083851482A3A3120B0FE47F08FEFDFC85F2
:100D0B001383851482A3A3E0F8A3E0F9A3E0FAA36D
:100D1B00E0FBC3120AF9400B851383851482E4F0C0
:100D2B00A304F074FF7FF8FEFDFC8513838514820A
:100D3B00A3A3E0F8A3E0F9A3E0FAA3E0FBD3120A24
:100D4B00F9500B85138385148274FFF0A3F0851380
:100D5B0083851482E0FEA3E0FF4E7003020FB9EF10
:0A0D6B00F47002EEF46003020E546F
:100D7500900012120B96E025E02466F582E4340318
:100D8500F583E0FEA3E0FFE4FCFD90000E120B9658
:100D9500120B0FE47F01FEFDFC90000E120B96E096
:100DA500F8A3E0F9A3E0FAA3E0FBC3120AF9500D9A
:100DB50090000E120B96120B1B0000000190001202
:100DC500120B96E025E02409F8E6FE08E6FFE4FCB0
:100DD500FD7BFF7A0FF9F8120AAA90000E120B9606
:100DE500E0F8A3E0F9A3E0FAA3E0FB1236139000C4
:100DF50006120B96120B0F900012120B96E075F06F
:100E050002A424ABF582E5F03402F583E0FEA3E00D
:100E1500FFE4FCFD900006120B96E0F8A3E0F9A3B1
:100E2500E0FAA3E0FB120AAA90000A120B96120B35
:100E35000FE47BFF7A0FF9F890000A120B96E0FC9D
:0C0E4500A3E0FDA3E0FEA3E0FF123613C3
:100E5100020F7A851383851482E0FEA3E064014EBC
:050E61006003020F8D8B
:100E6600900012120B96E025E02409F8E6FE08E64B
:100E7600FBAA06C374FF9BFF740F9AFEE49400FD61
:100E8600E49400FCE47BFF7A0FF9F8120AAA9000BA
:100E960006120B96120B0F900012120B96E025E02D
:100EA6002466F582E43403F583E0FEA3E0FBC37415
:100EB600FF9BFF740F9EFEE49400FDE49400FC90FB
:100EC600000A120B96120B0FE47F01FEFDFC900048
:100ED6000A120B96E0F8A3E0F9A3E0FAA3E0FBC33D
:100EE600120AF9500D90000A120B96120B1B000005
:100EF6000001900006120B96C083C082E0FCA3E0BE
:100F0600FDA3E0FEA3E0FF90000A120B96E0F8A313
:100F1600E0F9A3E0FAA3E0FB123613D082D08312E5
:100F26000B0F900012120B96E075F002A424ABF59D
:100F360082E5F03402F583E0FEA3E0FBC374FF9B79
:100F4600FF740F9EFEE49400FDE49400FC900006FE
:100F5600120B96E0F8A3E0F9A3E0FAA3E0FB120A6D
:100F6600AAE47BFF7A0FF9F8123613C374FF9FFFCA
:100F7600740F9EFE900012120B96E025E02409F8ED
:070F8600A60608A607D20928
:100F8D00900012120B96E0FF75F002A424ABF582CF
:100F9D00E5F03402F583E0FCA3E0FDEF25E02466E7
:0C0FAD00F582E43403F583ECF0A3EDF0D2
:060FB900900013020B7210
:03000000020800F3
:03000300021A03DB
:03000B00021A06D0
:03001300021A09C5
:03001B00021A0CBA
:03002300021A0FAF
:03002B00021A12A4
:03003300021A1599
:03003B00021A188E
:03004300021A1B83
:03004B00021A1E78
:03005300021A216D
:03005B00021A2462
:03006300021A2757
:03006B00021A2A4C
:03007300021A2D41
:10080000E4F5D9E5EF7480F5FF7402F5EF787FE445
:10081000F6D8FD9000007F007E08E4F0A3DFFCDE48
:07082000FA75812102086254
:1008270002128EE493A3F8E493A34003F68001F247
:1008370008DFF48029E493A3F85407240CC8C333D2
:10084700C4540F4420C8834004F456800146F6DFA1
:10085700E4800B010204081020408090341EE47EDF
:10086700019360BCA3FF543F30E509541FFEE49396
:10087700A360010ECF54C025E060A840B8E493A35D
:10088700FAE493A3F8E493A3C8C582C8CAC583CA88
:10089700F0A3C8C582C8CAC583CADFE9DEE780BE40
:01349100003A
:1008A700E709F608DFFA8046E709F208DFFA803E33
:1008B70088828C83E709F0A3DFFA8032E309F60820
:1008C700DFFA8078E309F208DFFA807088828C8388
:1008D700E309F0A3DFFA806489828A83E0A3F6083C
:1008E700DFFA805889828A83E0A3F208DFFA804C16
:1008F70080D280FA80C680D4806980F280338010ED
:1009070080A680EA809A80A880DA80E280CA803355
:1009170089828A83ECFAE493A3C8C582C8CCC583CD
:10092700CCF0A3C8C582C8CCC583CCDFE9DEE7809D
:100937000D89828A83E493A3F608DFF9ECFAA9F01C
:10094700EDFB2289828A83ECFAE0A3C8C582C8CC72
:10095700C583CCF0A3C8C582C8CCC583CCDFEADE8B
:10096700E880DB89828A83E493A3F208DFF980CCED
:1009770088F0EF60010E4E60C388F0ED2402B404E6
:100987000050B9F582EB2402B4040050AF2323458D
:0609970082239008F773B3
:10099D00BB010689828A83E0225002E722BBFE0258
:0909AD00E32289828A83E493228B
:1009B600BB010CE58229F582E5833AF583E02250F6
:1009C60006E92582F8E622BBFE06E92582F8E22240
:0D09D600E58229F582E5833AF583E493225A
:1009E300BB010689828A83F0225002F722BBFE01F3
:0209F300F322ED
:1009F500F8BB010DE58229F582E5833AF583E8F038
:100A0500225006E92582C8F622BBFE05E92582C8E3
:020A1500F222CB
:100A1700EF8DF0A4A8F0CF8CF0A428CE8DF0A42EF3
:020A2700FE22AD
:100A2900BC000BBE0029EF8DF084FFADF022E4CCB1
:100A3900F875F008EF2FFFEE33FEEC33FCEE9DEC7A
:100A4900984005FCEE9DFE0FD5F0E9E4CEFD22EDC0
:100A5900F8F5F0EE8420D21CFEADF075F008EF2F0A
:100A6900FFED33FD4007985006D5F0F222C398FDFB
:050A79000FD5F0EA2298
:100A7E00C5F0F8A3E028F0C5F0F8E5821582700203
:060A8E001583E038F022A0
:100A9400A3F8E0C5F025F0F0E58215827002158315
:060AA400E0C838F0E82272
:100AAA00E88FF0A4CC8BF0A42CFCE98EF0A42CFCEB
:100ABA008AF0EDA42CFCEA8EF0A4CDA8F08BF0A469
:100ACA002DCC3825F0FDE98FF0A42CCD35F0FCEBC8
:100ADA008EF0A4FEA9F0EB8FF0A4CFC5F02ECD398D
:0F0AEA00FEE43CFCEAA42DCE35F0FDE43CFC22FA
:10361300C2D5E830E70FB2D5E4C39BFBE49AFAE4E2
:1036230099F9E498F8EC30E717B2D5123649120C41
:103633000BE4C39BFBE49AFAE499F9E498F880035A
:10364300120C0B30D50DE4C39FFFE49EFEE49DFDF9
:04365300E49CFC22D5
:100AF900EB9FF5F0EA9E42F0E99D42F0EC6480C874
:060B090064809845F02213
:0C0B0F00ECF0A3EDF0A3EEF0A3EFF02259
:100B1B00A8828583F0D083D082120B32120B321253
:100B2B000B32120B32E473E493A3C583C5F0C58378
:100B3B00C8C582C8F0A3C583C5F0C583C8C582C824
:010B4B002287
:100B4C00D083D082F8E4937012740193700DA3A338
:100B5C0093F8740193F5828883E47374029368604C
:060B6C00EFA3A3A380DF4C
:100B7200E5142582F582E5133583F583B5130485E3
:100B820082142210AF06858214F51322858214F591
:040B920013D2AF22A9
:0D0B9600E5142582F582E5133583F58322F1
:100BA300EF4E6012EF60010EEDBB010B89828A8369
:100BB300F0A3DFFCDEFA2289F05007F709DFFCA976
:0C0BC300F022BBFEFCF309DFFCA9F022CD
:100BCF0075F008758200EF2FFFEE33FECD33CDCCDD
:100BDF0033CCC58233C5829BED9AEC99E582984060
:100BEF000CF582EE9BFEED9AFDEC99FC0FD5F0D63D
:100BFF00E4CEFBE4CDFAE4CCF9A88222B800C1B967
:100C0F000059BA002DEC8BF084CFCECDFCE5F0CBA4
:100C1F00F97818EF2FFFEE33FEED33FDEC33FCEBDD
:100C2F0033FB10D703994004EB99FB0FD8E5E4F998
:100C3F00FA227818EF2FFFEE33FEED33FDEC33FC85
:100C4F00C933C910D7059BE99A4007EC9BFCE99A79
:100C5F00F90FD8E0E4C9FAE4CCFB2275F010EF2FBE
:100C6F00FFEE33FEED33FDCC33CCC833C810D707BE
:100C7F009BEC9AE899400AED9BFDEC9AFCE899F8F9
:0E0C8F000FD5F0DAE4CDFBE4CCFAE4C8F9228C
:00000001FF
